:100000009AC30000B5C30000B3C30000B1C3000031
:10001000AFC30000ADC30000ABC30000A9C3000024
:10002000A7C30000A5C300000C944B290C94332AED
:100030000C9400299DC300009BC3000099C30000DD
:1000400097C3000095C3000093C3000091C3000054
:100050008FC300000C9427298BC3000089C30000C4
:1000600087C3000085C3000083C3000081C3000074
:100070007FC300007DC300007BC3000079C3000084
:1000800077C3000075C3000073C3000071C3000094
:100090006FC300006DC300006BC3000069C30000A4
:1000A00067C3000065C3000063C3000005010902C7
:1000B000A10185020901A1000509190129081500FE
:1000C0002501950875018102050109300931158165
:1000D000257F95027508810609381581257F9501D0
:1000E00075088106050C0A38021581257F95017572
:1000F000088106C0C005010980A101850319012AF4
:10010000B700150126B700950175108100C0050CD8
:100110000901A101850419012AA002150126A002E6
:10012000950175108100C005010906A1018506052C
:100130000719E029E71500250195087501810205D9
:1001400007190029EF1500250195F07501810205B9
:10015000081901290595057501910295017503910D
:1001600001C00660FF0961A1010962150026FF00B8
:100170009520750881020963150026FF00952075FA
:10018000089102C005010906A101050719E029E748
:1001900015002501950875018102950175088101F9
:1001A0000507190029FF150026FF0095067508812F
:1001B000000508190129051500250195057501910E
:1001C00002950175039101C00000000000000000CD
:1001D000000000000000000000000000000000001F
:1001E0000000000000000000000000007E0F00D4AE
:1001F000FFFFFFC7000000780000000000000000C3
:100200002A2B280000000000000000000000000071
:1002100000000029000000002C1E3420212224347C
:100220002627252E362D3738271E1F20212223244E
:1002300025263333362E37381F0405060708090AEA
:100240000B0C0D0E0F101112131415161718191A86
:100250001B1C1D2F3130232D350405060708090A04
:100260000B0C0D0E0F101112131415161718191A66
:100270001B1C1D2F3130354C09025B00030100A00F
:10028000FA09040000010301010009211101000124
:10029000224400070581030800010904010002034C
:1002A000000000092111010001222200070582033C
:1002B00020000107050303200001090402000103D7
:1002C00000000009211101000122B6000705840386
:1002D000200001120100020000000842534B5001AF
:1002E00000010203011C037600690061006C003A02
:1002F00000660036003400630032006200330063A1
:100300000000001003500061006E00630061006B8C
:100310000065000000120353007000610063006577
:10032000006D0061006E0000000403090429001440
:10033000001A000800150017001C0018000C00121D
:100340000013002A00225204001600070009000AC8
:10035000000B000D000E000F0033003400E1001D03
:10036000001B0006001900050011001000360037C0
:1003700000380031002B002D002E00E300E0002C9F
:10038000001E7CE200215223522F0030000100D1D8
:1003900000CD00D2000100010001004B0052004ED0
:1003A00000010001000100CF00CE00D000010001DB
:1003B000004A00500051004F004D0001000100DDD7
:1003C00000DE00DF0001000100010001000100016A
:1003D0000001000100010001000100010001000115
:1003E0000001000100010001000100010035001EB4
:1003F000001F0020002100220023002400250026E9
:1004000000270001000100010001000100010001BE
:1004100000010001000100010001000100010001D4
:1004200000010001000100010001000100010001C4
:1004300000010001000100010001000100010001B4
:100440000001000100010001000100010001003A6B
:10045000003B003C003D003E003F004000410042A8
:100460000043000100010001000100010001000142
:1004700000010001000100440045000100010001ED
:100480000001000100010001000100010001000164
:100490000001000100010001000100010001000154
:1004A0000001000100010001000100007C010001C9
:1004B000001603AB14FF140000020002001203AB8D
:1004C00014FF140000030001001703AB14FF140015
:1004D0000004000200FC02AB14FF146307050001D6
:1004E000001803AB14FF14000006000200FE02AB6C
:1004F00014FF140000070002001403AB14FF1400E3
:1005000000090002000003AB14FF146C070A00028C
:10051000000203AB14FF146C070B0002000403ABD2
:1005200014FF146C070C0002000603AB14FF146CDC
:10053000070D0002000803AB14FF146C070E000245
:10054000000A03AB14FF146C070F0002000C03AB8E
:1005500014FF146C07100002000E03AB14FF146CA0
:1005600007110002001003AB14FF146C0712000205
:10057000001A03AB14FF140000130002001C03ABAD
:1005800014FF140000140001001E03AB14FF14003C
:10059000001500000000009107650F000016000123
:1005A000001903C21416150000170001011903C237
:1005B0001416150000180001021903C214161500C4
:1005C00000190002002003AB14FF1400001A000100
:1005D000031903C214161500001B0002002203AB0E
:1005E00014FF140000FD377A585A000004E6D6B410
:1005F000460200210116000000742FE5A3E001E986
:1006000000DE5D003D8889C65436C3174FE4F9EC1F
:1006100072727025FA98E2F3FB7BF856EABCC9A027
:10062000249B37CEA08A9152F3FC0745501339E141
:100630007693723ABB304616D14760E1B349F4E88D
:100640005186B1E42657ECBD63982B39BCB647DC24
:100650006B258F09CDDACEED98311F16F25FAB3ED8
:1006600010A4FCD31A0A13124021B45C94DEC9E52D
:100670000EF4A25AC452C1E2CEE5914E5BE065BFD2
:10068000BD5EF54E980893BF718FA72DC59D23D9E8
:10069000C41FCDBDAF2C6EA673E79E74C39A34877A
:1006A0006EB0E6AF92106BEB82AF47216D4477924C
:1006B000915725C2E2B8C9CD0FD205B2ABD754B11C
:1006C00011729B481F196FBADBC7DFCF00AE0AF863
:1006D000414F3A45173B2A2FA776922152BA374B02
:1006E0007700000000CA551BAEEA6B6F960001FA56
:1006F00001EA03000017D8B8F1B1C467FB0200009B
:10070000000004595A4C4C4C4C4C4C2A52525252F8
:10071000524C4C4C4C4C4C2A52525252524C4C4C17
:100720004C4C4C2A52525252524C4C4C4C4C4C0059
:1007300052525252520011241FBECFEFDAE0DEBFF8
:10074000CDBF11E0A0E0B1E0E8E5F7E502C005901B
:100750000D92A03BB107D9F723E0A0EBB1E001C0B7
:100760001D92A932B207E1F70E94E4220C94592BA2
:1007700047CC9C01FB019A9581159F4120F5832F61
:100780008170B32FB270AA27732F74706627532F0E
:100790005870442734FF0DC08295807FAB2B09F041
:1007A0008062672B09F08064452B09F08068099509
:1007B0000895AB2B09F08260672B09F08460452B0C
:1007C000B1F38860F4CF80E0F2CF282F92959F702C
:1007D000963099F060F4925F9F70923030F4203F31
:1007E000B1F038F481E0283E38F080E008959A5F57
:1007F000F3CF81E0243FC9F7089591E0813F09F0EC
:1008000090E081E0283E08F080E0892B089581E0A7
:1008100008958093B00208958093B102089521E075
:1008200030E001C0220F8A95EAF78091B102822B55
:10083000F3CF21E030E0A90102C0440F551F8A9593
:10084000E2F7CA0180959091B1028923E5CF292F63
:10085000943090F58C3080F590E03CE0239F800D43
:10086000911D1124282F277041E001C0440F2A95C3
:10087000EAF723E0969587952A95E1F7FC01EE0FBC
:10088000FF1FE80FF91FEE57FD4F20E030E070E04A
:100890005191DF01CB01022E02C0969587950A94F3
:1008A000E2F7817081958527842385278E932F5FBA
:1008B0003F4F2330310561F70895292F943078F5A3
:1008C0008C3068F590E03CE0239F800D911D112451
:1008D000682F677023E0969587952A95E1F7FC01CC
:1008E000EE0FFF1FE80FF91FEE57FD4F40E050E0FD
:1008F00080E0219130E0062E02C0369527950A94BB
:10090000E2F721703327042E01C0220F0A94EAF780
:10091000822B4F5F5F4F4330510559F7089580E0B8
:1009200008959091B10221E030E0F90101C0EE0F8D
:100930008A95EAF7D90102C0AA0FBB1F6A95E2F7B0
:10094000EA2B01C0220F4A95EAF7892F8E23E8137C
:1009500003C0892F822B60CF2095822F8923FBCF64
:100960008091810290E020E0022E001C00082817F0
:1009700009060CF008952F5FF7CFFC01DB0184819D
:10098000813041F514968C911497813019F591813D
:100990008CE0E081F0E0899FE00DF11D1124EB5F18
:1009A000F84F94919A32B1F011962C911197EC91E5
:1009B000F0E0829FE00DF11D1124EB5FF84FE49110
:1009C00081E09E1301C080E091E0EA3209F090E0FE
:1009D000892B089581E008959C018091B2028D7960
:1009E000811119C0211540E5340780F4211580E2FA
:1009F0003807C0F42333310511F1D0F481E02E31F2
:100A0000310590F42430310530F00895C901965530
:100A10008115914010F080E00895C901805F9645EE
:100A20000797C8F33327E6CF2C323105A1F7089595
:100A30002653310981E02330310538F3ECCF81E0D2
:100A400008958091BC029091BB02981301C0089553
:100A50008F5F8770FACF9091B6028095892380933B
:100A6000B602282F2770211110C0891771F09091BC
:100A7000250392FF0AC0869586958695DADE109248
:100A8000B6021092B8021092B7020895982F90956E
:100A90008091B20289238093B20208958091AE02C0
:100AA000811531F01092AE021092AD021092AC029C
:100AB0000895803E9105D9F1C8F48133910509F478
:100AC00082C048F48932910509F472C08A329105D6
:100AD00009F480C0089589339105E9F082389105C1
:100AE000D1F08533910509F45EC00895843E9105E7
:100AF000D9F148F4823E910539F1833E910549F1DF
:100B000081EE90E00895863E9105C9F1873E9105FA
:100B100009F43EC00895209124032370211164C07C
:100B20002091250323FF14C089E290E008952091CD
:100B3000240320FD45C03091250330FF09C024FD6A
:100B400024C083EE90E008952091240322FDF7CF86
:100B500008952091240322FD44C03091250330FDE7
:100B600043C024FFF5CF11C02091250321FFF0CF12
:100B70008091240384FD09C087EE90E008952091C0
:100B8000240323FFE5CF24FFF7CF80E090E0089512
:100B90002091240323FD2BC03091250331FFE1CFA9
:100BA00084EE90E008952091240325FFD1CFBCCF9F
:100BB0002091240325FD1EC02091250323FFC8CFCB
:100BC00089E390E008952091240326FFC1CF8AE2B3
:100BD00090E008952091240326FFBACF81E390E0AE
:100BE000089582EE90E0089580EE90E0089586EEFC
:100BF00090E0089585E390E008959091240392FF9A
:100C000010C041E0282F2471243009F040E031E089
:100C1000282F2871283009F030E0431711F02CE01C
:100C2000822793FF10C041E0282F2471243109F05E
:100C300040E031E0282F2871283109F030E04317D7
:100C400011F02CE082273091250330FF10C051E0D5
:100C5000282F2171213009F050E041E0282F287120
:100C6000283009F040E0541711F029E0822731FFC5
:100C700010C041E0282F2171213109F040E031E01E
:100C8000282F2871283109F030E0431711F029E0AE
:100C9000822794FD877E08951F93CF93DF9309DF0A
:100CA000EC01811522E5920708F052C0811540E55C
:100CB000940708F0CDC0803E910520F58D3C91054C
:100CC00008F0A1C0883A910570F4853A910508F0C2
:100CD00097C081309105B9F10497813A910598F157
:100CE000C0E0D0E030C0885A91094B97C8F7C85A85
:100CF000D0E0CC0FDD1FCC5BDE4F0990D881C02D3A
:100D0000D46421C0811550E49507B0F4C11580E288
:100D1000D80708F0B3C0C83ED105A8F0CE019A9517
:100D200081159F41E8F68D2F68DF182FCE01992796
:100D3000C0DEEC01D12B07C09927BBDECC27DF70CA
:100D4000C82BD92BD06ACE01DF91CF911F91089586
:100D5000803842E59407C8F5803652E5950708F0DB
:100D60005BC0C03482E5D807D0F4C03292E5D90721
:100D700008F04BC08C2F8695869520E2829FC0019B
:100D80001124C37021E030E0A90102C0440F551FB7
:100D9000CA95E2F7EA01C82BD92BDD68D4CF8C2F96
:100DA00086958695877050E2859FC0011124C37097
:100DB00021E030E0A90102C0440F551FCA95E2F7B7
:100DC000EA01C82BD92BDC68BECF803C52E59507E1
:100DD00058F48F71C03AD245A0F590E0982F88273B
:100DE000EC01C46FD06AAFCF805C9245809708F069
:100DF00077CFDC2FCC27CC27DF71C06FD06AA3CF91
:100E0000A497D064A0CFD0659ECFCF71D0E0DC2F67
:100E1000CC27C16FD06A97CF86958695877020E2E0
:100E2000829FC0011124C37021E030E0A90102C0FB
:100E3000440F551FCA95E2F7EA01C82BD92BDA688F
:100E400082CFDBDEC82FD0E0DC2FCC27D0627BCF77
:100E50008F71D3DE93E0CC0FDD1F9A95E1F7CC279D
:100E6000DF70282F30E084FF05C050E1859F90019E
:100E700011243327C22BD32BD06965CF8D2F8F71CF
:100E8000BCDE182FCE01992714DEEC01D12BDECF6A
:100E900080E00895F894E82FE295EF70F0E041A12A
:100EA0008F7021E030E0B90102C0660F771F8A958C
:100EB000E2F7CB01962F9095942391A392A1892BD1
:100EC00082A3789408958091FC029091FD02909302
:100ED0001101809310010895ECEFF2E08481958177
:100EE0002AE030E0B9010E947E2A609314018681D5
:100EF000809315018285809303018485809302018C
:100F000086859785B9010E947E2A609312018089A7
:100F10008093130182898093010184898093000169
:100F20000895EF92FF920F931F93CF93DF93FB01EE
:100F30008FEF9FEF4430510508F45FC040912403C8
:100F400041FB882780F990E0880F991F42FB00271A
:100F500000F910E0000F111F000F111F802B912BC3
:100F600040FBEE24E0F8F12C8E299F2943FB222739
:100F700020F9C22F50E0D52F53E0CC0FDD1F5A953A
:100F8000E1F78C2B9D2B44FB222720F950E1259F74
:100F900090011124822B932B45FB222720F950E24C
:100FA000259F90011124822B932B46FB222720F9A9
:100FB00050E4259F90011124822B932B47FB22277D
:100FC00020F940E8249F90011124822B932B20913B
:100FD0002503322F3170932B26952170B22FBB0F32
:100FE000A0E08A2B9B2B092E000CAA0BBB0B808345
:100FF0009183A283B38380E090E0CDB7DEB7E6E0D3
:101000000C94DA2AAC0123E0969587952A95E1F7AE
:101010008E719927FC01E650FE4F0190F081E02D82
:101020004F70552721E030E002C0220F331F4A9550
:10103000E2F7611541F0E22BF32B86509E4FDC0165
:10104000ED93FC93089520953095E223F323F5CF9B
:10105000282F35EB2303C001112497FF04C08058CB
:101060009109892F089580589F4FFBCF8091960258
:10107000609104037091050380FF14C02091030167
:10108000269FC001279F900D1124BC01769567957E
:101090007695679560387105F0F561157105E9F190
:1010A000862F089581FF0BC020910301269FC00168
:1010B000279F900D1124BC0176956795EBCF82FF99
:1010C00009C0809103019B01829FB001839F700D35
:1010D0001124E0CF809195028115E1F290910201F7
:1010E00020910301891738F0CB01289FB001299F77
:1010F000700D1124CFCF289F90011124269FA001AD
:10110000279F500D369F500D1124692F70E0CA01A2
:101110000E947E2ABFCF8FE7089581E008958091D5
:10112000960280FF0CC06091010170E07595679593
:10113000759567956115710549F1862F089581FFB1
:1011400006C06091010170E075956795F3CF6091DD
:10115000010182FD0BC0909194029115A1F0609164
:10116000000180910101961738F0682F70E0603817
:10117000710500F38FE70895899FC001112470E085
:101180000E94922AF4CF61E070E0D7CF81E0089509
:10119000E0916702F0916802309739F00190F08198
:1011A000E02D309711F00995089580E00895A3E0AF
:1011B000B0E0EDEDF8E00C94C22A9C018091F801BA
:1011C0009091F90182179307B1F03093F9012093C0
:1011D000F801E0916702F0916802309761F00084B5
:1011E000F185E02D309739F083E089833B832A83B2
:1011F000CE01019609952396E2E00C94DE2AA3E045
:10120000B0E0E5E0F9E00C94C22A9C018091F6017F
:101210009091F70182179307B1F03093F701209373
:10122000F601E0916702F0916802309761F0008466
:10123000F185E02D309739F084E089833B832A8360
:10124000CE01019609952396E2E00C94DE2A909156
:101250001801913091F0A4EBB1E0EFEF90E02D9107
:10126000821751F0EF3F19F4211101C0E92F9F5F60
:101270009630A9F7EF3FC9F408959091240397FFA2
:10128000EACFE82FE695E695E695803FA8F7F0E0EF
:10129000E654FE4F877021E030E001C0220F8A95AE
:1012A000EAF78281822B828308950E2E000CFF0BB9
:1012B000EE54FE4FF8CF90911801913021F49091A7
:1012C000240397FD0CC0E4EBF1E09191891302C077
:1012D000DF011E9251E0EA3BF507B9F70895E82FC8
:1012E000E695E695E695803FC8F7F0E0E654FE4FB8
:1012F000877021E030E0A90102C0440F551F8A9594
:10130000E2F7CA01809592818923828308958091B2
:10131000170108952FB7F8948091F2019091F3018D
:10132000A091F401B091F5012FBF08958091FE02C4
:101330009091FF02892B89F0EDDF2091AC02309172
:10134000AD02AC01421B530B9A0181E04091FE02B9
:101350005091FF022417350708F480E00895CF93D9
:10136000DF93C091B2028091B502C82B8091AE028A
:101370008115E1F08091FE029091FF02892B19F016
:10138000D5DF81118BDBD091AE02809118018130C5
:1013900021F48091240387FD0DC086E024EB31E029
:1013A00090E0815058F4911179DBCD2B8C2FDF9197
:1013B000CF9108958EE12CEB31E0F2CFF90141910C
:1013C0009F01411571F39F5FECCF962F209125036C
:1013D00022FF0EC0682F660F660F660F692B6093A1
:1013E000B6021DDA97DF9093B8028093B702089592
:1013F00016CA9091AE02292F2823211559F0809505
:1014000089238093AE02811531F084DF8093AC0292
:101410009093AD02089580E090E0F8CFCF93C82F6D
:101420008091250382FF0BC08091AE028C1739F0AA
:1014300071DF9093AD028093AC02C093AE02CF9166
:10144000089568DF2091990230919A02232B21158B
:1014500021F080932F029093300220919B023091D3
:101460009C02232B211521F080932D0290932E02B4
:10147000E0916702F0916802309759F00680F78199
:10148000E02D309731F082E08093970287E992E077
:1014900009950895611509F441C0E3E3E80FE331CC
:1014A00048F4F0E0E55AF44D0C94A52ADFDD81956F
:1014B00080939A02C6CFDADDFBCFD8DD8195809389
:1014C0009902F8CFD3DDFBCF2ADE80939B02F2CFC7
:1014D00026DE8195FACF23DE819580939C02EACFA8
:1014E0001EDEFBCF815D990B21E030E001C0220FB1
:1014F0008A95EAF780919802822B80939802DACF3E
:1015000080919602816080939602D4CF809196025A
:101510008260F9CF809196028460F5CF4091990264
:101520008D3C59F480919A0287FF0DC010929A0267
:10153000411559F41092950208C08E3C81F48091B7
:101540009A0218169CF3411581F080919B029091AC
:101550009C02892B8111AECF10929402ABCF8F3CAD
:1015600041F447FFF0CF1092990280919A028115C1
:10157000E0CF803D19F41416B4F3E5CF90919B02AF
:10158000893D29F41916FCF610929B02DCCF8A3DA6
:1015900019F497FFD8CFF8CF90919C028B3D29F496
:1015A00097FFD1CF10929C02CECF8C3D19F4191623
:1015B000CCF3C9CF9FE2980F983090F4815D990BDE
:1015C00021E030E0B90102C0660F771F8A95E2F78B
:1015D000CB01809590919802892380939802B3CF94
:1015E0008D3D31F4809196028E7F80939602ABCF31
:1015F0008E3D21F4809196028D7FF7CF8F3D09F0CB
:10160000A2CF809196028B7FF0CF2FB7F894609194
:10161000F2017091F3018091F4019091F5012FBFD7
:10162000089587E797E7909301088093000888E181
:101630009AE00FB6F894A895809360000FBE90933F
:101640006000FFCFFC019B018091E8019091E901CE
:101650008617970740F0672B29F48091E8008E7772
:101660008093E800C90140E0009741F4411106C0B1
:101670008091E80082FF2FC080E008952091400211
:101680002115A9F12530A9F12091E80023FD2DC0F5
:101690002091E80022FDECCF2091E80020FFE4CF6C
:1016A0003091F3002091F200009719F028303105B5
:1016B00058F041E02830310509F040E02091E80081
:1016C0002E772093E800D0CF41914093F10001970D
:1016D0002F5F3F4FE9CF80914002811541F0853067
:1016E00041F08091E80083FFC3CF81E0089582E05C
:1016F000089583E008958091E20187FF13C08091EF
:10170000E80082FF06C08091E8008B778093E800B4
:101710000895809140028111F2CF08958091400296
:101720008115D9F38091E80080FFF8CF8091E8001F
:101730008E77ECCF2091E4003091E50095E6A90189
:101740002091EC00822F817020FF06C08091E8007C
:1017500080FF06C080E008952091E80022FD1AC0B5
:1017600080914002811589F0853089F08091EB00ED
:1017700085FD0FC02091E4003091E500421753072A
:10178000F9F29A95E1F684E0089582E0089583E005
:10179000089581E00895E8EDF0E080818E7F8083F8
:1017A0001092E2001092DA001092E100A0EEB0E098
:1017B0008C9181608C9380818F77808319BCA7ED99
:1017C000B0E08C918E7F8C9380818F7E808310928D
:1017D000E1010895E0916702F0916802309739F0D5
:1017E0000284F385E02D309711F060E209950895A9
:1017F000982F9093E900891771F07091EC00209177
:10180000ED005091F00021FD09C09F5F973089F7EE
:101810008093E9000895762F242F50E03091EB005B
:101820003E7F3093EB003091ED003D7F3093ED0033
:101830003091EB0031603093EB007093EC0020931B
:10184000ED005093F0002091EE0027FDDECF0895CB
:10185000A0E0B0E0EEE2FCE00C94BC2AC8EDD0E0E1
:1018600088818F7E8883E7EDF0E0808181608083CE
:1018700084E082BF81E08093E10188818E7F88834C
:1018800002EE10E0F80110821092DA0081EEC82E0C
:10189000D12CF601108288818F77888388818068B7
:1018A000888388818F7D888319BC109240021092B2
:1018B000E001109223021092DF0190EEE92EF12C4C
:1018C000F70180818B7F808388818160888342E0FB
:1018D00060E080E08DDFF60180818E7F8083F801FB
:1018E000808181608083808188608083F70180812E
:1018F0008E7F8083888180618883CDB7DEB7E8E002
:101900000C94D82AE091BC029091BB0227E0E91325
:1019100002C080E00895AE2FB0E02E9FF0011124A8
:10192000E354FD4F3181361306C03081381303C0B4
:101930003581341304C0FD013196E770E8CF81E0B2
:1019400008959C012115310509F408958FE99FE060
:101950000197F1F700C0000021503109F3CF0F9338
:101960001F93CF93DF938B01EA0190914002943053
:1019700051F58093E9008FEF9091E80095FD06C046
:1019800095ED9A95F1F700008A95B1F78091E800FE
:1019900085FF19C0CFDE811111C08091E80085FD5F
:1019A00006C08091E8008E778093E800F3CFF801BD
:1019B00081918F018093F100219779F78091E80060
:1019C0008E778093E800DF91CF911F910F9108955A
:1019D000792F603229F440E250E0682F82E0BFCFD7
:1019E0000895CF93DF93D82FC92F48E050E0682F98
:1019F000792F81E0B4DF88E0ED2FFC2FAAEEB1E073
:101A000001900D928A95E1F7DF91CF910895BC0185
:101A100040E250E084E0A3CFBC0146E050E084E027
:101A20009ECFBC0143E050E084E099CF9091250324
:101A300092FB222720F9281771F080FB92F99093EE
:101A40002503609124037091250384E090E00E94B7
:101A5000452B82E000C808951F93CF93DF93962F04
:101A6000122F632F282F292B2430C8F44C30B8F4C0
:101A7000C42FD0E0CC0FDD1F28E1929FC00DD11DF7
:101A8000112490E6899FC00DD11D1124CE018996A5
:101A90000E942B2B612FCE018A960E942B2BDF9167
:101AA000CF911F91089580911801813061F5809147
:101AB000240387FF28C053DC8093BB0140E250E041
:101AC00067E472E08AEB91E00E94F22A892BD1F060
:101AD00080E2EAEBF1E0A7E4B2E001900D928A9592
:101AE000E1F7E0916702F0916802309759F00480C5
:101AF000F581E02D309731F086E08093BA018AEBD2
:101B000091E0099508952BDC8093B20148E050E004
:101B100069E672E082EB91E00E94F22A892B91F350
:101B200088E0E2EBF1E0A9E6B2E001900D928A953F
:101B3000E1F7E0916702F0916802309719F30280B3
:101B4000F381E02D3097F1F282EB91E0DACF81154D
:101B500031F09091B202892B8093B202A4CF089504
:101B6000811531F09091B502892B8093B5029BCFFE
:101B70000895811519F00E94460595CF08958115A5
:101B800039F080959091B50289238093B5028BCF6F
:101B90000895CF93C82F8115C1F08CEF8C0F813A37
:101BA00080F580911801813021F48091240387FD14
:101BB0000EC0E4EBF1E08191C817F9F021E0EA3BB7
:101BC000F207C9F78C2F43DB6EDFCF910895EC2F1E
:101BD000E695E695E695F0E0E654FE4F828190E0CA
:101BE0004C2F477021E030E002C0220F331F4A958E
:101BF000E2F782239323892B29F38C2F5CDB53DFBD
:101C0000E1CF80E28C0F883068F4C77081E090E00B
:101C100001C0880FCA95EAF7C091B202C82BC093E1
:101C2000B202D2CF8BE58C0F833030F42C2F2452AC
:101C3000330BC901BCDAC9CFE8E5EC0FEB3148F44E
:101C4000F0E0EE0FFF1FE658FE4F80819181D7DA5A
:101C5000BCCF83E38C0F833108F0B7CF61E08C2FCA
:101C600019DCB3CFCF93DF93EC01805E9109089725
:101C700020F060EB7DE0209711F467EA7DE0CE0173
:101C80000E94B9038C2F85DFDF91CF9108956115F4
:101C900029F02091B50222602093B5029C013052B8
:101CA0002115304308F49927DDCF811541F19CEFD0
:101CB000980F913A10F4FFDAF6CE90E2980F983030
:101CC00050F4877091E001C0990F8A95EAF7892F47
:101CD0000E944605F1CF9BE5980F933018F480E001
:101CE00090E065CA98E5980F9B3118F480E090E089
:101CF00086CA93E3980F933110F460E0CBCB08953C
:101D0000CF93DF93EC01D1DFCE01805E910908977C
:101D100020F06FEB7DE0209711F469EB7DE0CE01C0
:101D20000E94B903DF91CF9108951F93CF93DF9362
:101D3000182FEB012EDF209731F4812FB6DFDF91D2
:101D4000CF911F9108958FE99FE00197F1F700C0AF
:101D500000002197F0CF60911C0370911D0389331F
:101D600021F060911A0370911B03DFCFEF92FF9275
:101D70000F931F93CF93DF93C62FD42F122F81156C
:101D800099F06093AA02C6DA9093DE018093DD0198
:101D9000C77081E001C0880FCA95EAF7D8DECDB7D9
:101DA000DEB7E6E00C94DA2A8091AA0268132DC00F
:101DB000E090DD01F090DE01ADDA8E199F09883CDC
:101DC000910518F500E20D0FCD1799F0C770FF24AB
:101DD000F3948F2D01C0880FCA95EAF7CADE083048
:101DE00040F48D2F877001C0FF0C8A95EAF78F2D84
:101DF000AEDE812FB0DF083090F6D77081E001C0F1
:101E0000880FDA95EAF7B5DECACFC77081E001C066
:101E1000880FCA95EAF7F7CF1092B20280911801A5
:101E2000813011F58091240387FF1EC0ECEBF1E0B7
:101E30008EE1DF011D928A95E9F780E090E0B7D945
:101E400080E090E0DCD91092B5022DDE86E0E7E973
:101E5000F2E0DF011D928A95E9F710929502109247
:101E6000940210929602EDCAE4EBF1E086E0E1CF35
:101E7000D3DF2FEF84E39CE0215080409040E1F7D6
:101E800000C0000088E19AE00FB6F894A89580930E
:101E900060000FBE90936000FFCFCF93DF93D82FE9
:101EA000C92F20918102283010F0B6DF20E0E22F08
:101EB000F0E0EE0FFF1FEF58FD4FD083C1832F5F7F
:101EC00020938102DF91CF910895CF93DF93FB019F
:101ED0008FEF9FEF44305105B0F0D081C1819CDF7E
:101EE000D0932403C370809125038C7FC82BC093AB
:101EF0002503609124037091250384E090E00E9403
:101F0000452B80E090E0DF91CF910895AAE2B0E008
:101F1000ECE8FFE00C94C12A82EE91E0FC0101960E
:101F20002091F100208321E08A3E9207B9F7809149
:101F3000E301893009F457C0C8F4823009F4B2C013
:101F4000833009F482C0813081F18091E80083FF01
:101F5000E6C08091E2019091E3019A3008F0DFC081
:101F6000E92FF0E0E259F44D0C94A52A8A3009F4E7
:101F700089C08B3051F78091E201813231F7809135
:101F8000E6019091E701892B01F78091E800877FB6
:101F90008093E800B0DB81E09091E401911101C0F1
:101FA00080E08093180138DFD0CF8091E201813A40
:101FB00061F68091E800877F8093E8008091E601D8
:101FC0009091E701892B59F060E080E090E070E0AB
:101FD00039DB8091E8008B778093E800B6CF68E02A
:101FE0008AEE91E0F4CF8091E201813209F0ADCF29
:101FF0008091E6019091E7018D7F892B09F0A5CFB3
:102000008091E800877F8093E8008091E80082FF5C
:1020100017C09091F3008091F200029731F4809103
:10202000F100813011F0863021F48091F10080932D
:1020300017018091E8008B778093E8005CDB85CF07
:10204000809140028111E1CF80CF8091E201813AFD
:1020500009F07BCF8091E6019091E701892B09F08F
:1020600074CF8091E800877F8093E8008091E8003A
:1020700080FFFCCF809118018093F1008091E800EF
:102080008E77DACF8091E201813209F05ECF8091C4
:10209000E800877F8093E8002EDB8091E501809344
:1020A000160153CF8091E201813A09F04ECF809121
:1020B000E800877F8093E8008091E80080FFFCCFF4
:1020C00080911601D9CF803889F0823841F580910E
:1020D000E6018F70873018F58093E9008091EB005E
:1020E00085FB882780F91092E90006C080912302C1
:1020F000880F9091DF01892B9091E800977F909352
:10210000E8008093F1001092F1008091E8008E7752
:1021100023C0811116C08091E401813009F18091C2
:10212000E80083FF0AC08091E800877F8093E80081
:102130008091EB0080628093EB00AA96E3E00C9420
:10214000DD2A823061F78091E401811581F01092DF
:10215000E9008091E800877F8093E800CCDADFCF48
:1021600081E0933009F080E080932302F0CF8091EA
:10217000E6018F702FEF280F263088F68093E90054
:102180002091EB0020FFE3CF933031F48091EB00FE
:1021900080628093EB00DBCF9091EB009061909395
:1021A000EB0021E030E0A90102C0440F551F8A95E1
:1021B000E2F74093EA001092EA008091EB00886019
:1021C000E8CF8111ACCF1091E4011F778091E3003B
:1021D0008078812B8093E3008091E800877F809353
:1021E000E80089DA8091E80080FFFCCF8091E3006D
:1021F00080688093E30083E0111101C082E0809346
:1022000040028DCF8058823008F089CF8091E40160
:102210009091E5018C3D53E0950791F583E08A8329
:102220008AE289834FB7F894DE01139620E03EE0FE
:1022300051E2E32FF0E050935700849120FF03C058
:1022400082958F703F5F8F708A30C0F0895C90E01C
:102250008D939D932F5F243161F74FBF8091E800EC
:10226000877F8093E8006AE270E0CE010196EAD9A8
:102270008091E8008B778093E80051CF805DE7CFB5
:10228000292F33272330310509F44EC078F521304A
:10229000310509F488C08BE590E0E8E7F2E02230F0
:1022A000310509F03CCF2091E800277F2093E8001A
:1022B0002091E8013091E9018217930708F49C010D
:1022C00040E02115310509F073C0411171C08091C2
:1022D000E80082FDCDCF80914002811549F2853022
:1022E00039F28091E80083FFF2CFC2CF8091E601FE
:1022F0009091E7012132310509F446C022323105BF
:1023000009F00DCF8330910508F009CFFC01EE0FE5
:10231000FF1FE85DFE4F0190F081E02D8B5D9E4F29
:10232000DC018C9190E010C09C013327823021F1B8
:102330002330310568F4232BB9F4E9E2F3E0E491AA
:102340008E2F90E0E9E2F3E0009709F4E8CEABCFFE
:102350002330310509F0E3CEE5EEF2E0E4918E2F73
:1023600090E0E5EEF2E0F0CFE5E1F3E0E4918E2FCE
:1023700090E0E5E1F3E0E8CFE3E0F3E0E4918E2FD5
:1023800090E0E3E0F3E0E0CF8330910508F0C7CEC2
:10239000FC01EE0FFF1FE25DFE4F0190F081E02D8A
:1023A00089E090E080CF82E190E0E3EDF2E07BCF46
:1023B00080914002811509F45BCF853009F458CF34
:1023C0008091E80083FD54CF8091E80082FD7FCFAB
:1023D0008091E80080FF75CF9091F3008091F2002A
:1023E0002115310519F08830910550F041E008972A
:1023F00009F040E08091E8008E778093E80061CF9B
:1024000044914093F1003196215031090196E8CF73
:10241000803809F084CE8091E800877F8093E800BF
:102420008091E0018093F10070CE811178CE1091FF
:10243000E401123008F073CE8091E800877F80932A
:10244000E8001093E00157D91115D9F084E080938A
:10245000400242E061EC81E0CBD942E261EC84E0F1
:10246000C7D942E261EC82E0C3D942E260EC83E08A
:10247000BFD980914002843051F482E080931901E9
:102480004ECE8091E30087FDE1CF81E0E0CF81E097
:10249000F5CF80911A01877F80931A019091B50240
:1024A0009D7F9093B50284FF08C08F7E80931A01B0
:1024B0008091B20282608093B20280911A0185FFFE
:1024C00008C08F7D80931A018091B2028062809350
:1024D000B202E9CACF92DF92FF920F931F93CF937C
:1024E000DF93EC018B01F42E80911A0182FF61C011
:1024F000C090A102D090A202CC16DD0619F0209760
:1025000009F057C080911A018B7F80931A01C1E0B6
:1025100081FD10C080919F029091A0029801281B1C
:10252000390BC1E0809110019091110128173907F2
:1025300008F4C0E080911A01C0FB81F980931A0170
:102540006C2FC6010E9402088091B20281FF08C070
:1025500080911A01806180931A0182E00E944605F1
:102560008091B20285FF08C080911A018062809339
:102570001A0180E20E9446056C2FC60188DBF11427
:1025800031F08091170385FF02C086FF25C080913E
:102590001A0390911B03D5D98091A1029091A202B8
:1025A0009C0130522115304308F49927A9DB71DFD3
:1025B0000FC0CE01905281159043B0F4CE019927FF
:1025C0009FDB8091A1029091A202C817D90779F3ED
:1025D0001093A00200939F02DF91CF911F910F9162
:1025E000FF90DF90CF900895CE01EACF0F931F9315
:1025F000CF93DF930CEF12E0C9EAD1E0CE010E9445
:102600000F2BF80161918F01681719F0CE010E941C
:102610002B2B2196C13DF1E0DF0781F7DF91CF91B0
:102620001F910F9108950F931F93CF93DF930CEF9A
:1026300012E0C9EAD1E0CE010E940F2BF80181938C
:102640008F012196C13DF1E0DF07A9F7C7EBD4E088
:10265000FE0185919591009711F0FC0109952C964A
:10266000F5E0CF3EDF07A1F7DF91CF911F910F91EA
:102670000895ECEFF2E0128E138E8FEA90E09183D2
:10268000808325E0248F88E893E1938382838AE026
:1026900090E09583848344E150E05783468348E08B
:1026A00050E051874087938782876EE170E075879D
:1026B00064879787868780E590E0918B808B538B2A
:1026C000428B48E250E0558B448B42E350E0578BFD
:1026D000468B48EC50E0518F408F158E55A344A394
:1026E000178E168E91A380A322A317A216A27EDFB7
:1026F00093DB109225031092240380E08460809382
:10270000250360E074E084E090E00E94452B8BCFCD
:102710008F929F92AF92BF92CF92DF92FF920F93D0
:102720001F93CF93DF9380903E0290903F0281E011
:1027300090E090933F0280933E02A12CB12C00E0E8
:10274000650110E012C0FE01259135914F2D612FDA
:10275000802F82D92296F3948CE0F812F4CF8CE08B
:10276000C80ED11C1F5F143039F0E601CC0FDD1FFD
:10277000C35DDC4FF12CE7CF0F5F80E3A80EB11CE7
:102780000430F1F676DF90923F0280923E02DF91B4
:10279000CF911F910F91FF90DF90CF90BF90AF909E
:1027A0009F908F9008950F931F93CF93DF93982F4F
:1027B000962B943020F54C3010F5C42FD0E0CC0F80
:1027C000DD1F28E1629FC00DD11D112430E6839FDB
:1027D000C00DD11D1124CE0189960E940F2B082F08
:1027E00010E0102F0027CE018A960E940F2B98012F
:1027F000282BC901DF91CF911F910F91089580E09F
:1028000090E0F8CF462F672F209143023091440289
:10281000232B81F4703F39F4403F61F480914102F1
:10282000909142020895982F972B943018F44C30D1
:1028300008F4B9CF80E090E00895A0E0B0E0E3E2D2
:10284000F4E10C94BD2A7C010091B1028091B002A8
:10285000082BC3E0D0E010E0C8010C2E02C0959513
:1028600087950A94E2F780FD09C02197A8F7D12C3B
:102870008D2DCDB7DEB7E7E00C94D92ADC2EB70159
:102880008C2FC0DF0E944C06019779F3F1CFCF93D4
:10289000DF93D82FC92FD1DF6D2F7C2FB3DF0E949C
:1028A0004C06DF91CF910895FC018481811529F0B8
:1028B00080819181ECDF0C94E50380E008951F9303
:1028C000CF93DF93182FD92F611589F0411579F037
:1028D000B4DFC82F682F812F9D2F0E942704612FFE
:1028E0007D2F8C2F8FDFDF91CF911F9108950E9454
:1028F0005D04C82FF4CFFC01462F65818081918152
:10290000DECF382F292FCB01A32FB22F8F3222E019
:102910009207A105B10520F48F529E4F0C940F2B06
:1029200080E0089585E290E00E940F2B8D3B89F4B2
:1029300086E290E00E940F2B8A3459F487E290E0FF
:102940000E940F2B91E0863F09F090E0892F817063
:10295000089580E0FCCF9C01CB01BA01F9013296C9
:10296000E4914E2F50E06E17710548F0F90134964E
:10297000659175910E94FF2A80E090E008958FEFA5
:102980009FEF0895A4E0B0E0E8ECF4E10C94BF2AD6
:102990008B01FC013396F49019821A821B821C82EF
:1029A000452B31F48FEF9FEF2496E5E00C94DB2A62
:1029B00044E050E0BE016F5F7F4FCDDF019691F3A1
:1029C00081E090E00F2C02C0880F991F0A94E2F773
:1029D000092E000CAA0BBB0B49815A816B817C81AB
:1029E00084239523A623B72321E0892B8A2B8B2BC5
:1029F00009F420E0F801208380E090E0D5CF9C012D
:102A0000CA01F9013296E4914E2F50E08E179105DC
:102A100050F0F9013496859195910E94FF2AE6DDE8
:102A200080E090E008958FEF9FEF0895A4E0B0E07C
:102A3000ECE1F5E10C94BB2A7C016B01CA01F701C2
:102A40003396B49019821A821B821C82892B31F42E
:102A50008FEF9FEF2496E9E00C94D72A44E050E0F2
:102A6000BE016F5F7F4FC70176DF019689F381E07A
:102A700090E00B2C02C0880F991F0A94E2F7809512
:102A80009095092E000CAA0BBB0B49815A816B81D2
:102A90007C8184239523A623B723F6012081022F6E
:102AA000017010E00B2C02C0000F111F0A94E2F716
:102AB000012E000C220B330B802B912BA22BB32B5E
:102AC00089839A83AB83BC8344E050E0BE016F5F8F
:102AD0007F4FC70194DFBECFA8E0B0E0E2E7F5E1A9
:102AE0000C94B62AFE01319688E0DF011D928A958A
:102AF000E9F794E3A92E91E0B92E8F013F01EE246E
:102B0000E394F12C34E4C32E31E0D32EF50181910E
:102B10005F018F3F09F444C0F894E82FE295EF700D
:102B2000F0E021A18F70A70102C0440F551F8A95C4
:102B3000E2F7CA01922F982B91A392A18095892345
:102B400082A3789400C0E8E3F1E021E030E0812C3A
:102B5000912C41914F3F79F0A42FA295AF70A05EC8
:102B6000B0E08C9190E04F7002C0959587954A95A2
:102B7000E2F780FF3BC080E090E0882A992A220F8C
:102B8000331FCE16DF0629F7F50182918F3F11F032
:102B90000E944A0750EA5A95F1F7D8018D929C920B
:102BA0000E5F1F4FB8E3AB16B1E0BB0609F0AECF26
:102BB00048E050E0B3018AE192E00E94F22A892BBA
:102BC000B9F088E0F301AAE1B2E001900D928A9594
:102BD000E1F781E08093DC010E948A099093DB0198
:102BE0008093DA012896EEE00C94D22AC901C5CF71
:102BF0008091DC018115B1F30091DA011091DB01C4
:102C00000E948A09801B910B059760F348E050E011
:102C10006AE172E086E392E00E94F22A892B49F091
:102C200088E0EAE1F2E0A6E3B2E001900D928A9535
:102C3000E1F71092DC01D6CFA0E1B0E0E2E2F6E1EC
:102C40000C94B42AFE01319680E1DF011D928A9531
:102C5000E9F703E210E091EDA92EBB24B3942FE233
:102C6000422E22E0522E612C712C4F017301620121
:102C7000B1E14B165104610471041CF080E1C82ECF
:102C8000D12CA601B501C4010E941C2BAC0CBD1CAB
:102C90000D2C000CEE08FF084C185D086E087F082C
:102CA0000150104019F76096E0E10C94D02A6FEFC4
:102CB00085E290E00E942B2B6FEF86E290E00E946D
:102CC0002B2B6FEF87E290E00E942B2B60E088E2D5
:102CD00090E00E942B2B1CDDAFDF6DEB85E290E0D6
:102CE0000E942B2B6AE486E290E00E942B2B66EF79
:102CF00087E290E00C942B2BA0E0B0E0E2E8F6E154
:102D00000C94BB2AEC0188818115E9F0813009F02F
:102D100041C08981813021F48A8123961CD8F3CF68
:102D2000823029F48A8123960E94C90DECCF83302A
:102D300029F48A8123960E94550EE5CF843041F014
:102D400022968111E0CFCDB7DEB7E9E00C94D72A07
:102D50008A81239620E030E09AE0682F6053770B59
:102D6000AB016A30710560F02115310551F3EFE9CF
:102D7000FFE03197F1F700C0000021503109F4CF96
:102D8000929FB001939F700D11249A01260F371F57
:102D90008991E3CFE82FF0E0E850FE4FB490282F60
:102DA00026952695269530E0F901E851FE4FE490EE
:102DB0008770F12C082E02C0F594E7940A94E2F78C
:102DC000E0FAEE24FF24E0F8F901E852FE4FC49047
:102DD000D12C082E02C0D594C7940A94E2F7C0FA09
:102DE000CC24DD24C0F8F901E853FE4F049110E033
:102DF00002C0159507958A95E2F701701127E11435
:102E0000F10419F081EE0E94C90DC114D10419F02A
:102E100086EE0E94C90D60E070E08B2D0E94950E39
:102E2000C114D10419F086EE0E94550EE114F1048C
:102E300019F081EE0E94550E0115110519F08CE272
:102E40000E94AB0E21965FCFA8E0B0E0EAE2F7E186
:102E50000C94B22A8C01FC018481811509F4A0C272
:102E600060E0C80148DD9C01F8018681803170F482
:102E70004091BC029091BB02491331C09091FA027B
:102E8000911521F09091FB02903148F1F801958164
:102E9000911110C02115F0E53F0708F085C02115FC
:102EA00040E2340708F095C0283E310588F4203E02
:102EB0003105A8F430939E0220939D02F80182818F
:102EC00093819093BA028093B90210921B0107C0BC
:102ED000C9019A9581159F4168F72111EBCF61E0F7
:102EE000C80109DD7C01F8018581811509F400C163
:102EF000C70197578038910508F0FAC0BE2CF0E161
:102F0000EF1608F03DC26EE272E080E090E0F9DC7E
:102F1000811136C2C12CD12C7601B1105CC044E0C5
:102F2000242EAE014F5F5F4F58874F83EF81F885A6
:102F3000222D11922A95E9F7460157013FEF831A96
:102F4000930AA30AB30AC701B601DBDC89838115A2
:102F500009F416C2813009F0C7C02601370142E0EA
:102F6000440E511C611C711CC501B401CADC382E11
:102F70008A83811509F404C28FEF830D833008F032
:102F80003EC0C301B201BDDC8B83811519F0CE01B7
:102F90000196B2DE4601570153E0850E911CA11C3B
:102FA000B11C75016401C2CF203E82E5380760F490
:102FB000203892E5390708F092CFC9018052924536
:102FC000809708F077CF8BCFC90187579C4702972E
:102FD000F8CF8031F6CF2FE2C21622E0D206E1040C
:102FE000F10409F4CDC1C701B6018BDC3FEFC31A70
:102FF000D30AE30AF30A8111EECFBA948ECF8BEF96
:10300000830D8330E0F54601570183E0880E911C63
:10301000A11CB11CC301B20174DC8B83811509F4BE
:10302000C0CFC501B4016DDC8C83811108C046019D
:10303000570194E0890E911CA11CB11CB2CFAB804A
:10304000BC80E1E0AE16EFEFBE0610F0BA2CAA2469
:10305000F6E03F1681F027E0321649F0C5010E94E4
:10306000A32280911A0390911B030E94A10CC50119
:103070000E94C422DCCFC5010E94A322D8CF34E035
:103080005301420133128DCFC301B2013ADC782ED5
:103090004601570144E0840E911CA11CB11CC701DC
:1030A000B6016D5F7F4F8F4F9F4F2BDC711409F47A
:1030B00067C1811509F464C18150990B4FEF489F96
:1030C0009001499F300D1124E72DE150FF0B2E0F89
:1030D0003F1F2150310908F464CF8FE99FE0019729
:1030E000F1F700C00000F5CFCE01019605DE59CF03
:1030F0008091170380FFBCC00E948A095C01F8011F
:103100008581811509F4C5C080911A0182FF05C02F
:1031100040E0B50180E090E0DDD9F4E1EF16FCE796
:10312000FF0609F4B2C025E1E2162CE7F20609F425
:103130004AC033E1E3163CE7F30609F48CC0C7014B
:1031400090528115904308F047C01092A20210924D
:10315000A102F801958191111092AA02F6E1EF16F1
:10316000FCE7FF0609F064C18091B20230911603BA
:1031700030FF04C0282F247421114EC1282F2A7A31
:1031800031FF04C0482F4171411120E032FF04C0DB
:10319000482F4878411120E033FF03C0827281112B
:1031A00020E0911509F43AC181E0211101C080E0CD
:1031B0008093AB0285E3211101C089E20E942709B7
:1031C0000E94530DDDC090911A01892F8E7F90FFD0
:1031D000816080931A015DD980911A0180FF48C0F7
:1031E000F8E2EF16F10408F06CC02EE1E216F104EB
:1031F00008F07CC0C70104974A9790F580911703A7
:1032000084FD2EC0F8018581811509F4E3C09091F9
:10321000B2028091AE02D82ED92A2D2D2D7F2115F4
:1032200009F469C01092A2021092A1022091170322
:1032300021FD61C060E0C7010E94020860E0C70193
:103240000E94470E8091AE028D7F0E940E0A82E09E
:103250000E942B0595C080911A01816080931A010C
:10326000F8018581811521F01092A2021092A1022D
:10327000F8018581F701E851FC47E730F10508F0D6
:1032800068CFE858F44D0C94A52A80911A018E7FDE
:10329000A0CF80911A018F7E51EEE516F10439F02E
:1032A00085EEE816F10431F480911A018F7D809348
:1032B0001A0192CFC70190528115904308F08CCF2C
:1032C00048CF39E3E316F10468F44DE2E416F10463
:1032D00020F45BE2E516F10419F68091170382FDF4
:1032E000BFCF90CF84E6E816F104F6CF80911703A4
:1032F00083FDB6CF87CF27E0F801A3EAB2E00190C3
:103300000D922A95E1F71092A6021092A5028090E4
:10331000A1029090A202E814F90409F045C020919E
:10332000170325FF41C030911A0131FBCC24C0F8AE
:1033300031FF02C026FF38C020919F023091A002C9
:10334000A501421B530B483C510570F591FF08C085
:1033500080911A01806180931A0182E00E944605E3
:103360008091B20285FF08C080911A01806280932B
:103370001A0180E20E9446056C2DC4010E94470E8E
:103380008091B6028770811559F0F8018581811509
:1033900039F08091250382FF03C082E00E942B0553
:1033A0002896E2E10C94CE2A8D7F0E940E0AF092BC
:1033B000A202E092A102B092A002A0929F028D2DE3
:1033C0008270846090911A01997FD82ED92AD09268
:1033D0001A013DCF40E0B501C7017CD8D1CF26E22C
:1033E00041EE61EE0E94B60ECBCF27E245EE65EED0
:1033F000F9CF26E241EE60EEF5CF27E245EE64EE2E
:10340000F1CF26E241EE62EEEDCF27E245EE66EE29
:10341000E9CF28E241E0EBCF20E0B2CE8091AB02D1
:10342000811521F085E30E945B09CACE89E2FBCFBA
:1034300027E7E2162CE7F20609F138E7E3163CE746
:10344000F30639F19701205E32452032310530F51F
:1034500091113FC04E2D4F7181E090E0FC0102C000
:10346000EE0FFF1F4A95E2F77F016E2F83E090E099
:103470000E942B2B8E2D0E94090482CF81E0911592
:1034800051F00E940F0443E062E081E00E94910449
:1034900077CF82E0F4CF0E941904F5CF9115C9F0DF
:1034A000FAE5EF16FCE7FF0609F493C008F068C0E0
:1034B00031E0E3163CE7F30609F489C043E0E41683
:1034C0004CE7F40609F47DC0E1145CE7F50609F465
:1034D0006BC0F8018581C080D180811509F47DC061
:1034E000C601ABD9F82E682FC6010E942704B60189
:1034F0008F2D88D90E944C06F82ED92E86E0F8012F
:10350000DE01119601900D928A95E1F7F801C580D0
:10351000B680B2942FE0B2228091B60287708115F6
:1035200009F1AC2CC114F9F0892F807F803469F047
:1035300080E28F0D8830B0F0892F807E803229F4B0
:10354000F2E0FF1678F0B11469F08091250382FF54
:1035500009C082E00E942B058091B6028770AA24E0
:10356000A3948111A12C8D2D82958F70882E912C82
:103570008C3008F055C0F401E158F44D0C94A52AA4
:103580008BE5E8168CE7F80631F1809125030024DD
:1035900082FF0394802D9CE5E9169CE7F90609F06B
:1035A00098CF0E94160D95CF0E940C0FEFEFF4E319
:1035B0002CE0E150F0402040E1F700C000000E9404
:1035C000110B6FEF7FEF80E090E00E94452B0E948F
:1035D000380F81E0E6CF80E0E4CFC6010E945D04B1
:1035E000F82E85CF2D2D2F70E22E30E1D31618F056
:1035F000E29490EFE922C11409F44AC0E11469F0A1
:1036000080E28F0D883010F0F1103CC08091B20242
:103610008E298093B2020E94530D8F2D0E94C90DF6
:1036200048E0841A910854E08516910418F40E9429
:10363000C808A12C8F2D9D2D0E94E503811541F016
:10364000C11409F423C2B11409F417C2109228035B
:10365000A114A1F08091B60280FD10C0F80115827E
:103660008695869586950E940F04C801EDDB8091B2
:10367000B6028695869586950E94190460E0C80179
:103680003AD98ECE8091B5028E298093B502C3CFF0
:103690008F2D0E94550EE11419F280E28F0D8830B3
:1036A00010F0F11004C08E2D0E94460506C0E09473
:1036B0008091B5028E218093B5020E94530DB0CF48
:1036C0008D2D8F70E82E8D2D807F803219F0E29441
:1036D00080EFE822F11451F091E0F91609F475C079
:1036E000C11409F481C0B114E9F097CF809125038A
:1036F00082FD14C0C11459F0E11439F08091B20276
:103700008E298093B2020E94530D80E087CF80E023
:103710000E94550EE11409F483CFC5CFC11491F175
:10372000B11004C08E2D0E94A70D7ACFE1E0BE1229
:1037300011C07090AE028E2D8721E81609F470CF6B
:103740000E948A099093AD028093AC027E28709209
:10375000AE0266CF80911803823008F461CFB812B0
:103760005FCF8E2D0E94A70D8E2D0E94F9098091AA
:10377000AF029E2D9823E91609F452CF8E2980932B
:10378000AF024ECFB11012C08E2D0E94B90D8E2DFA
:103790000E94F9098091AF029E2D9823911509F49A
:1037A0003FCFE094E822E092AF023ACF8091180335
:1037B000823008F435CFF1E0BF1232CF8091B202EF
:1037C0008E21811509F42CCFDFCF80911E03C11407
:1037D00021F08B1508F424CFA5CFB81608F020CF20
:1037E0008E2D0E94B90D1CCFB114D1F329E3F2162E
:1037F00009F03BC180911C0390911D030E94A10C14
:103800008F2D0E94550E0CCF8D2D86958695837039
:10381000811569F0813009F003CF8F2D9D2D9370B4
:10382000C11002C080E090E00E94FF08F9CE8F2D09
:103830009D2D9370C11002C080E090E00E94D708D7
:10384000EFCE6C2D8F2D0E944A0AEACE8D2D83700B
:10385000811133C0C110E4CE4F2D4295469547707B
:10386000440F440F8F2D8F70042E01C0880F0A94CF
:10387000EAF72F2D2071F4FE07C02FE030E001C0E1
:10388000220F4A95EAF720953D2D369536953370EF
:10389000323071F0333051F04091B002313029F0C4
:1038A000822B84230E940904BBCE842B822BFACF67
:1038B000822B9091B0028927F5CFC11459F1D0FE27
:1038C000AFCE4F2D429546954770440F440F8F2D34
:1038D0008F70042E01C0880F0A94EAF72F2D2071F3
:1038E000F4FE07C02FE030E001C0220F4A95EAF74E
:1038F00020953D2D369536953370323089F0333032
:1039000069F04091B102313041F0822B84230E9452
:103910000C0486CE8230A8F683CE842B822BF7CF80
:10392000822B9091B1028927F2CF3D2D3F70E32E7B
:10393000C11429F0832F0E940F048F2DF4CE8F2DF8
:103940000E94B90D8E2D0E9419046ACE42EFF41622
:10395000A1F153EFF51670F480EFF816D1F091EF66
:10396000F91691F0C11409F47BC0B11056CE8D2D1B
:103970008F7127C0E3EFFE1639F1F4EFFF12F2CF9B
:103980008091250382FD2CC08D2D8F71C114D9F239
:1039900018C080911E03C11461F0B81608F040CE23
:1039A0002D2D2F7181E090E001C0880F2A95EAF754
:1039B000B8CF8B1508F434CEF3CF8D2D8F71C11095
:1039C000C2CF0E940F042CCE80E0C11409F49FCF17
:1039D00081E09D2D9F7101C0880F9A95EAF797CFDE
:1039E00080911803823048F1C114C9F09091B60259
:1039F0009770943059F41092B6021092B802109257
:103A0000B7028D2D8F710E94190411CE63E0B81694
:103A100008F00DCE8D2D8F710E94E50908CEB816E5
:103A200040F01092B6021092B8021092B70264E011
:103A3000F1CF81E00E942B05FACDC11431F063E093
:103A40008D2D8F710E94E509EBCD81E00E942B0541
:103A500022E0B21608F4E4CD82E00E942B05E0CD0E
:103A6000B11441F039E3F316C3CE80911A0390915B
:103A70001B03C4CE8D2D8F7166CF8091B4028093CD
:103A8000B3028091B2028093B402E2CD40E060E0E4
:103A900089819A810E945F149C01E090B202B11466
:103AA00029F010922803E092B402D2CD809126032F
:103AB0009091270328173907B1F78091190382FFE6
:103AC000F0CF80912803811561F38091B3020E94A9
:103AD000A70D8F2D0E94AB0E8091B3020E94B90DED
:103AE000E0CF8091FB02803178F48091FA02811559
:103AF00059F0E091BC022091BB023091F602409156
:103B0000F50257E02E1301C008956E2F70E05E9FFE
:103B1000F0011124DF01A354BD4F14968C9114972A
:103B2000811551F111968C911197831325C08C91B9
:103B3000841322C015968C91159781111DC0129681
:103B40008D919C91A091F702B091F8028A1B9B0B7A
:103B5000883C910588F48091FB028F70806180938E
:103B6000FB02ED53FD4F80818F708061808385EF74
:103B700092E06AD90C942105FB013196E770C2CF1F
:103B8000CF92DF92FF920F931F93CF93DF93182F63
:103B9000092F87E0F82EC091BC028091BB02C817A4
:103BA00091F1FC9EE0011124CE0183549D4F6C01E4
:103BB000FC018581811589F0C6010E94541481158C
:103BC00061F0FE01ED53FD4F20812F7020612083B5
:103BD000F601808191810E944D0FC60135D9209157
:103BE000BC0230E02F5F3F4F277033272093BC0289
:103BF000C354DD4F89818013CECF88818113CBCF11
:103C00008D81811541F2DF91CF911F910F91FF902E
:103C1000DF90CF900895EF92FF921F93CF93DF93A1
:103C2000EC0120911B01211541F010E0812FDF9163
:103C3000CF911F91FF90EF900895EA80FB80E61AE4
:103C4000F70A24EFE21621E0F20678F760E0CE01F1
:103C50000E947B149C0130522115304330F70E94A2
:103C6000EC04811511F380919D0290919E020E94B7
:103C7000EC04182F8115C9F280912203909123033F
:103C8000853F21E0920710F084EF91E0E816F906F5
:103C900060F68E818F7080618E83888199810E9409
:103CA0004D0F0E94B004CE01CFD8C0CFADE0B0E040
:103CB000ECE5FEE10C94B42A8C0186E0F801DE010B
:103CC000189601900D928A95E1F7D8016C901196A3
:103CD0005C9011971296AD90BC9013971496EC904F
:103CE00014971596FC90F1100CC050918102252F6D
:103CF00030E0E0E08E2F0E2E000C990B8217930718
:103D00003CF155EFC52E52E0D52E8091F90281117C
:103D100051C0E114D1F0F11409F401C3C8010E94AB
:103D20005414811509F4FBC26091B9027091BA0272
:103D3000C80171DF811109C087E0F801A5EFB2E089
:103D400001900D928A95E1F7CCDEFF24F39485C0B3
:103D5000880F991F8F589D4FDC0111964C91119738
:103D6000451103C08C91681611F0EF5FC3CFEF3F90
:103D700041F2D80116968C9116978F708061169635
:103D80008C93E517A0F4AFEFA50FA0938102EA177B
:103D900070F4F0E0EE0FFF1FEF58FD4FB0E0AA0FF8
:103DA000BB1FAF58BD4F8D919C91918380830E9422
:103DB000B004A7CF60E085EF92E00E947B149C01E5
:103DC0007090FA028091F7029091F8024501881AEA
:103DD000990A711409F450C2B8EC8B16910408F0DA
:103DE00009C2E11409F4B1CF8091F602F801918182
:103DF000E090FB02F0E1EF1608F0C5C198134FC048
:103E00009091F502D8018C91981349C0F11047C0E8
:103E10008E2D8F7080618093FB0285EF92E014D825
:103E20008091FB02F8018683F090F702E090F8029F
:103E300047E0D42E0091BC028091BB02081751F0DC
:103E4000D09E8001112403541D4FD80115968C91EA
:103E5000811108C00E942105F12C8F2D2D96E0E1E3
:103E60000C94D02AF801B280C380C8010E94541477
:103E700081110EC0C8010E9424178091BC0290E0FD
:103E80000196877099278093BC02FB2CEC2CD2CF33
:103E90006F2D7E2DC801BFDE8111EFCFDBCF3052F9
:103EA0002115304308F084C0F11005C140E0652DB4
:103EB000862D0E94820C81114FC040E0652D862D19
:103EC0000E94820CF82E811509F429C180911903F2
:103ED00080FFC2CF85EF92E00E94241760E085EF5B
:103EE00092E00E947B148C01F090BC027F2C98E041
:103EF000E92E25EF822E22E0922E37E0432E80918C
:103F0000BB027816A1F0A72CB12C479CC00111244C
:103F1000FC01E354FD4F6F0160E0CF010E947B1470
:103F2000582E692ED60115968C91811197C0B8E054
:103F3000EB1618F417E0EF10ACC08885998520DEE9
:103F40000E94B0040E94210587E0E5EFF2E0DF0166
:103F50001D928A95E9F780CF60E0C8010E947B142A
:103F60008091190383FFA9CFB80185EF92E00E94E9
:103F7000BD048111A2CF8091FB028F70806180937C
:103F8000FB028091F5029091F6020E944D0F85EFA1
:103F900092E00E942417E5EFF2E087E0DF011D9236
:103FA0008A95E9F788859985EBDD0E94B00452CFA8
:103FB000F11409F482CF8091FB0281608093FB02AF
:103FC0008091190381FF48CF85EF92E00E9424176A
:103FD0000091BC028091BB02081709F4CCC0E02E0E
:103FE000F12CB7E00B9FC0011124FC01E354FD4FFD
:103FF0006F01CF010E945414811509F4BCC087E001
:10400000F601A5EFB2E001900D928A95E1F7C701A4
:10401000019687709927082F8093BC020E94210582
:1040200087E0F82E8091BB02801709F413CFF09E31
:104030008001112403541D4FC8010E9454148111A2
:1040400009CFC8010E9424178091BC0290E001961C
:1040500087709927082F8093BC02E4CF1052011576
:10406000E0E31E0708F063CF8091190383FD0AC0C7
:10407000E72CC5010196F82FF7707F2E052D162D20
:1040800046013DCFB601C4010E94BD04811589F3EC
:10409000EFCF1F9DC001112483549D4F0E94241710
:1040A0002091BC0230E02F5F3F4F27703327F22E64
:1040B0002093BC0240CF8091FB0281608093FB0281
:1040C00060E0C8010E947B148091190383FF78CFC0
:1040D000B80185EF92E00E94BD04811171CFF0908C
:1040E000FB02E894F0F8F092FB02C8010E9454141D
:1040F0008111B2CE8F2D8F7080618093FB028091F1
:10410000F5029091F6020E944D0F0E94B00485EFD7
:1041100092E00E942417E5EFF2E087E018CF88854F
:1041200099850E944714292F22952F70903450F4BE
:104130009F70223080F0911599F0F80196819031AE
:1041400078F48BCE2A5F2F70223078F0C8010E945D
:104150002417F72C82CE911519F0811509F47DCE24
:10416000805E883008F479CEF1CF803F08F475CEB8
:10417000815F8330F7CF87E0E5EFF2E0DF011D924A
:104180008A95E9F74DCF981315C09091F502F80183
:10419000808198130FC0F1100DC0E682C8010E9403
:1041A000241787E0F801A5EFB2E001900D928A95FF
:1041B000E1F7CBCDC8010E945414811509F4AFC0BA
:1041C000F11409F4ACC08091FB02803208F4B4CD44
:1041D0008091F5029091F6029A838983BC82AB822A
:1041E0008091F9028D831E82EF82CE0101960E949A
:1041F0002417A2CD9090FB02F0E19F1638F485EFD2
:1042000092E00E94241787E0D601A2CEE11409F4BF
:104210009CCD9091F602F8018181981311C0909184
:10422000F502808198130CC0F1100AC09682C80173
:104230000E94241787E0D6011D928A95E9F785CD63
:10424000C8010E945414811509F469C0F11409F4DD
:1042500066C08091FB02803208F46ECD8091F50239
:104260009091F6029A838983BC82AB828091F90295
:104270008D831E829F82B9CFB8EC8B16910408F013
:1042800052C0E11409F461CDF11409F448C09091D1
:10429000F602F801818198132AC09091F50280817D
:1042A000981325C060E085EF92E00E947B14809116
:1042B0002003909121038816990608F072CF80910F
:1042C000FB0280FD6ECF803108F46BCFD8011696CB
:1042D0008C931697982F907F903F09F45FCF982F7B
:1042E000907F905F8F70892B16968C9357CFC80163
:1042F0000E945414811571F06091B9027091BA0254
:10430000C80189DC811509F417CD87E0E5EFF2E0FB
:10431000DF0192CF8091FB0281608093FB02C80194
:104320000E94241712CD87E0F60111928A95E9F7D1
:1043300093CDABE1B0E0EFE9F1E20C94BE2A4E8BF5
:104340005F8B688F798F082F8A8F192F9B8FF82E9C
:10435000E92E811509F4A1C040E0692F8E899F895B
:104360000E945F149C01111549F01092280390934C
:104370002703809326031092B5020AC0809126037A
:10438000909127038217930719F481E08093280303
:104390001D8A86E0FE017696DE011F9601900D9241
:1043A0008A95E1F78091250382FF21C08091FE026A
:1043B0009091FF02892BD9F00E948A092091B702BF
:1043C0003091B802821B930B2091FE023091FF02C4
:1043D0008217930738F08091B60282FD03C082E015
:1043E0000E942B050E94960981110E944E05F1142E
:1043F00061F00B8B1C8B61E0CE010F960E947B1449
:1044000061E0CE010F960E947B140B8B1C8B87E022
:10441000FE013F96DE01189601900D928A95E1F714
:10442000CE01089643DC811110C02091BB0230916F
:10443000BC0287E0FE013896DE01119601900D92D4
:104440008A95E1F78C8581112CC017E08091BC0220
:104450009091BB02891741F0189FC0011124835429
:104460009D4F24DC811144C08C85811112C0809144
:104470001B0181110EC08A859B852091B902309164
:10448000BA02821B930B8F3F9F4318F081E0809309
:104490001B016B96E6E00C94DA2A911509F478CFAB
:1044A0006ACF822F90E001968770992738171906F6
:1044B00071F40E940C0F1092BB021092BC0287E0B4
:1044C000E5EFF2E0DF011D928A95E9F7BECF97E0B4
:1044D000929FD0011124A354BD4FFE01319601904B
:1044E0000D929A95E1F78093BB020E942105ADCF12
:1044F0008091BC0290E00196877099278093BC025E
:10450000A5CFA6E0B0E0E7E8F2E20C94C02A0E9452
:104510008A098C018091450290914602801791078B
:1045200071F019821A820E948A09BC0149815A815C
:1045300080E090E0FEDE109346020093450226964E
:10454000E4E00C94DC2AA6E0B0E0E9EAF2E20C94A4
:10455000C22A9093420280934102811520E2920781
:1045600030F40E94320E2696E2E00C94DE2A80EFB0
:1045700089838A830E948A098160BC0149815A81AA
:1045800081E091E0D6DEEFCFA6E0B0E0E9ECF2E228
:10459000F9C79093420280934102811520E292076D
:1045A00030F40E94800E2696E2E00C94DE2A80EF22
:1045B00089838A830E948A098160BC0149815A816A
:1045C00081E090E0B6DEEFCFCDB7DEB7AC970FB6A7
:1045D000F894DEBF0FBECDBF85B7806885BF85B7B5
:1045E000806885BF84B7877F84BF0FB6F894A8958D
:1045F00080916000886180936000109260000FBE1F
:1046000080E890E00FB6F894809361009093610089
:104610000FBE81E08093190188E497E09093B10187
:104620008093B0010E9413130E94CB0B0E94280CB0
:104630008091E20084608093E2007894809140024F
:10464000811599F08091E9001091EC008F70179519
:1046500011271795182B1092E9008091E80083FD2F
:104660000E94860F1F701093E90082E084BD93E0E2
:1046700095BD9AEF97BD80936E000E9492148111B0
:1046800002C00E94571681E30E944A0783E30E94FA
:104690004A0782E30E944A0786E30E944A0708E32A
:1046A00011E0D8018D918D018F3F11F00E944A07D2
:1046B000B1E004341B07A9F788E0E6E3F2E0DF018C
:1046C000282F1D922A95E9F7EAE1F2E0DF011D9219
:1046D0008A95E9F780E090E0AAD7833E9E4F21F4C7
:1046E0000E949214811123C063EE7EEF80E090E07F
:1046F000CCD760E082E090E0AED781E08093B0025A
:1047000061E083E090E0A7D760E074E184E090E0AE
:10471000BCD70E94571640E050E0BA018FE090E00D
:10472000ACD740E050E0BA0183E190E0A6D782E048
:1047300090E075D78093240284E090E078D790933E
:104740002503809324030E946C15EFEFF6E721E028
:10475000E150F0402040E1F700C000000E946C15DD
:104760008091360280FF07C06FEF7FEF80E090E01E
:104770008CD70E94110B83E090E051D70E9409046E
:1047800084E091E090936802809367028E010F5F4E
:104790001F4F80914002853049F48091400285305E
:1047A00009F45EC00E940C0F0E94C8080E946C159C
:1047B000E5E26E2EE2E07E2EF6E3EF2EF2E0FF2E33
:1047C000D701F301219131918D919D914DE252E0FC
:1047D0004E175F0709F47AC02817390799F376E373
:1047E000872E72E0972E312CD401CD90DD904D01B3
:1047F000F301419051903F014C145D0451F14C2460
:104800005D24212CAA24A394B12CC2018A219B21CE
:10481000892BB1F029823A820E948A099C838B837A
:10482000F1E0FD8391E096012A213B21232B09F43D
:1048300090E09E8349815A816B817C818D8179DDF5
:104840002394AA0CBB1C2CE02212DFCFF301D292DE
:10485000C292339434E03312C7CF0E94050B3BC0A1
:1048600080914002843021F11092220248E150E010
:1048700080E40FB6F894A895409360000FBE809333
:10488000600083B7817F846083BF83B7816083BF0B
:104890007894889583B78E7F83BF0FB6F894A895D8
:1048A00080916000886180936000109260000FBE6C
:1048B0000E946C15E6E3F2E081919191892B09F059
:1048C00054C492E0EE33F907B9F767CF28173907D8
:1048D00009F085CF16DE8091170380FF1CC0809100
:1048E0001A0182FF18C00E948A09BC0180919F02B0
:1048F0009091A0029B01281B390B8091100190918F
:1049000011012817390738F041E08091A1029091F8
:10491000A2020E946A1286E0E7E9F2E0D801019063
:104920000D928A95E1F77090980290909902A0906C
:104930009A0280909B02B0909C0210929902109271
:104940009A0210929B0210929C028A2D892981154D
:10495000A1F0C0902F02D09030020E948A099C01E1
:104960002C193D0990919502911509F48DC0809103
:1049700015018217130608F495C08B2D882981151F
:10498000A1F0C0902D02D0902E020E948A099C01B5
:104990002C193D0990919402911509F4B3C08091AE
:1049A00013018217130608F4BBC080919802871187
:1049B00019C080919902811511F0891113C02091BD
:1049C0009A02211511F02A110DC090919C029115A7
:1049D00011F09B1107C030919B02311103C0822B53
:1049E000892B81110E94210A86E0F801A7E9B2E033
:1049F00001900D928A95E1F70E94C80890913102CA
:104A0000891721F0809331020E94050B80914002AA
:104A1000843009F0BECE83E08093E9008091E80005
:104A200082FFB7CE8091E80090E085FF0AC00E9427
:104A30009A0B40E2C42ED12C5801811509F4AAC06A
:104A400091E08091E8008B778093E800911509F45C
:104A5000A0CEC0904302D0904402E981C114D10499
:104A600009F4A6C0EE3F09F0C5C08A81833020F06A
:104A70008550833008F0BEC0EA81EE3008F0BAC03D
:104A8000F0E0E557F44D61C5409114018AE0489F7C
:104A9000A00111244217530708F06FCF9F5F909336
:104AA000950202C09F3FD1F7911459F00E94360839
:104AB00091E019140CF09FEF899F802D11248093B1
:104AC0009902A11459F00E94360891E01A140CF0D2
:104AD0009FEF899F802D112480939A0280919902E3
:104AE000811509F44ACFD0909A02D11409F445CF28
:104AF0000E942808809399028D2D0E942808809397
:104B00009A023BCF40911201AAE04A9FA0011124D2
:104B10004217530708F049CF9F5F9093940202C059
:104B20009F3FD1F7811459F00E948F0891E018142B
:104B30000CF09FEF899F802D112480939B02B1146C
:104B400059F00E948F0891E01B140CF09FEF899F91
:104B5000802D112480939C0280919B02811509F481
:104B600024CFD0909C02D11409F41FCF0E942808B2
:104B700080939B028D2D0E94280880939C0215CF64
:104B80008091F100F50181935F01F1E0CF1AD10826
:104B900009F456CF8091E80085FDF2CF8091E800BE
:104BA0008B778093E8000E949A0B811599F348CF88
:104BB000E43148F4E11551F0E150E33138F4F0E02C
:104BC000E756F44DC2C4EE3F09F456CF8FEFF9C259
:104BD0001A8289E08B830EC08A81823079F083301B
:104BE000A9F0813099F70E94050BB5D46B837C83C3
:104BF0008D839E83C8010E94EA0BCBCD88E290E0B2
:104C00000ED51B821C821D828E83F4CF80913E02C2
:104C100090913F02892B71F3F8018EE392E0D70166
:104C20002C9111963C91B2E0EB0EF11C3283238360
:104C300032968E159F0599F7DDCF8A81823031F645
:104C40006B817C818D819E8186D488E290E003D542
:104C5000D1CF4C816B818A810E94D31398278927F9
:104C600098279E838D83C6CF2D813E8132272327AF
:104C700032274C816B818A810E942C0DBBCF0E9410
:104C80008813B8CF80E18A83B5CF82E08A838FE230
:104C9000A1CF8C818D3108F0ADCF8A809B80982484
:104CA00089249824A12CB12C68017801E80EF11C0C
:104CB000EC14FD0409F49ECF80E0EFE28E16E2E0F2
:104CC0009E06A104B10420F4C4018F529E4FA7D4C4
:104CD000D60114968C93BFEFCB1ADB0AEFEF8E1A36
:104CE0009E0AAE0ABE0AE4CF80913E0290913F0236
:104CF000892B09F47FCF8C818D3108F07BCF482E32
:104D0000512C612C712CCA80DB80DC24CD24DC2466
:104D1000E12CF12C1801812C912C54018414950460
:104D2000A604B70408F066CFFFE2CF16F2E0DF0674
:104D3000E104F10438F4D10114966C91C6018F524C
:104D40009E4F89D4BFEF8B1A9B0AAB0ABB0AEFEFC9
:104D5000CE1ADE0AEE0AFE0AFFEF2F1A3F0ADECF56
:104D60000E941C1647CF84E08ECF8C818D3108F0D5
:104D700041CF482E512C612C712CCA80DB80DC2461
:104D8000CD24DC24E12CF12C812C912C54011E012A
:104D900025E0220E311C84149504A604B70408F003
:104DA00029CF80E030E8C31631E0D306E104F104F6
:104DB00018F4C601899633D4D1018D931D01BFEF3C
:104DC0008B1A9B0AAB0ABB0AEFEFCE1ADE0AEE0A79
:104DD000FE0AE1CF2C81E22EF12C2D3108F00ACF12
:104DE0008A819B819827892798272C01612C712C17
:104DF0008038F1E09F0708F0FDCE822E912CA12C87
:104E0000B12C40E851E060E070E0441955096609B2
:104E10007709421751056105710508F4EBCE209121
:104E20003E0230913F02232B09F03FC09C01275DD9
:104E30003F4F3CA72BA780FBCC24DD24C0F880FF8C
:104E40000BC08896ECD39D818927982789278115E7
:104E50009C4711F48FEF8D83D501C401840D951DFE
:104E6000A61DB71D80FF1AC0170141E0241A3108A2
:104E7000CE010596820D931D9AA789A78BA59CA5A7
:104E80008E0D9F1DCCD3A9A5BAA59C9181159C47D9
:104E900021F48FEFE9A5FAA580837101F801EC0DEB
:104EA000FD1D2FEFCE14DF0428F01801C12CD12CEA
:104EB000760126C09481858181159C4711F4248355
:104EC000258342E0C40ED11C3296ECCF50E8451643
:104ED00051E055066104710430F4D10114966C91CF
:104EE000C2018996B8D3BFEFCB1ADB0AEB0AFB0AE3
:104EF000EFEF4E1A5E0A6E0A7E0AFFEF2F1A3F0A84
:104F0000C814D904EA04FB0408F374CE80913E026D
:104F100090913F02892B09F46DCEC8010E94EA0BE3
:104F20002FEF31EE44E0215030404040E1F700C027
:104F300000001FCC88E0ECE1F1E0DE0191960190E9
:104F40000D928A95E1F7FE0132968FE1DF011D9205
:104F50008A95E9F786E0898388E07F96DE011596D9
:104F600001900D928A95E1F745CE80E2898381E038
:104F70008A831B821C823ECE8B819C81092E000C71
:104F8000AA0BBB0B35E0880F991FAA1FBB1F3A95D0
:104F9000D1F7AC01BD01405E5F4F6F4F7F4F4817A7
:104FA00059076A077B0708F425CE8032E1E09E07A7
:104FB000A105B10508F01ECE4132F1E05F076105A1
:104FC000710520F040E251E060E070E0481B590BB1
:104FD000BC016B517A4FC801FCD20CCE4AE150E0C3
:104FE0006FEF70E0CE01079613D380913E02898364
:104FF000CA821B821C821D828BE006CE81E090E07B
:10500000909344028093430282E390E090933502B0
:10501000809334020E948A09909333028093320273
:10502000E9CDC114D10481F1B0903602A0903702CD
:10503000E0903202F09033020E948A098E199F0993
:105040008536910540F1A3FE26C0B0FE24C00E9423
:105050008A099093330280933202809134029091B6
:10506000350201979093350280933402892B61F4C5
:10507000109244021092430281E090E090933F022C
:1050800080933E02C12CD12C80913E028983CA823A
:10509000809134029FCD82E390E09093350280931B
:1050A0003402F2CF10923F0210923E02A3CDEB8069
:1050B000FC8040E250E06FEF70E0C801A9D22DEA19
:1050C00034E042E050E080E090E0F90165917591B4
:1050D000E616F70630F4800F911FDC016D937C9388
:1050E000CA01B5E0293D3B0709F484CDAC014E5F10
:1050F0005F4F245F3F4F4132510538F37BCD2B8109
:105100003C818DEA94E0FC014591559124173507C7
:1051100009F448C00C96E5E0853E9E07A1F756CD00
:105120008B819C812DEAE22E24E0F22EF70125915D
:1051300035918217930709F446C0FCE0EF0EF11C8D
:1051400025EEE21625E0F20689F7CC24CA94DC2C81
:1051500055C00E9439134ECD8B8181114BCD80E219
:10516000D8011D928A95E9F745CD809123028115DA
:1051700009F413CBA0E1A9BDB2E1B9BD09B400FEA9
:10518000FDCF8091D8008F7D8093D8008091E00082
:1051900082608093E0008091E00081FDFCCF0E945E
:1051A0000C0FFBCAFC01369625913591211531056E
:1051B00009F40CCD4FE150E0BE016E5F7F4FF90165
:1051C0000995898317CDF7013896259135912115D9
:1051D000310509F4BACF4CE150E0BE016B5F7F4F5F
:1051E000C701F90109956C01892B41F4F7013A9641
:1051F00085919591009711F0FC010995C982FACC2F
:105200001F921FB61F9211248F939F93AF93BF934A
:1052100080912202811113C08091F2019091F301DB
:10522000A091F401B091F5014196A11DB11D8093AB
:10523000F2019093F301A093F401B093F501BF91B3
:10524000AF919F918F911F901FBE1F9018957894DA
:105250001F921FB61F9211248F939F93AF93BF93FA
:105260008091F2019091F301A091F401B091F501C8
:105270000196A11DB11D8093F2019093F301A093BB
:10528000F401B093F501BF91AF919F918F911F9061
:105290001FBE1F9018951F920F920FB60F921124E8
:1052A0002F933F934F935F936F937F938F939F932E
:1052B000AF93BF93EF93FF938091E10082FF09C00A
:1052C0008091E20082FF05C08091E1008B7F809396
:1052D000E1008091DA0080FF24C08091D80080FF37
:1052E00020C08091DA008E7F8093DA008091D9000F
:1052F00080FFA9C080E189BD82E189BD09B400FEBB
:10530000FDCF81E0809340028091E101811109C0CD
:105310000E94CB0B0E94280C8091E2008460809355
:10532000E2008091E10080FF1AC08091E20080FFDE
:1053300016C08091E2008E7F8093E2008091E200AF
:1053400080618093E2008091D80080628093D800D1
:1053500019BC85E08093400283E08093190180911D
:10536000E10084FF2FC08091E20084FF2BC080E128
:1053700089BD82E189BD09B400FEFDCF8091D800CE
:105380008F7D8093D8008091E1008F7E8093E10033
:105390008091E2008F7E8093E2008091E200816044
:1053A0008093E2008091E001811509F452C084E00D
:1053B0008093400280914002843009F052C082E024
:1053C000809319018091E10083FF2CC08091E2005D
:1053D00083FF28C08091E100877F8093E10082E015
:1053E000809340021092E0018091E1008E7F8093D3
:1053F000E1008091E2008E7F8093E2008091E200E4
:1054000080618093E20042E060E080E00E94F80B5F
:105410008091F00088608093F00081E08093190112
:1054200080931801FF91EF91BF91AF919F918F9160
:105430007F916F915F914F913F912F910F900FBE90
:105440000F901F90189519BC109240021092E10124
:1054500068CF8091E30087FF02C083E0A9CF81E09D
:10546000A7CF81E0ADCF1F920F920FB60F921124FC
:10547000EF92FF920F931F932F933F934F935F935E
:105480006F937F938F939F93AF93BF93CF93EF933C
:10549000FF9309EE10E0F8018081C091EC008F705D
:1054A000C795CC27C795C82B108280EFE82EF12C2A
:1054B000F7018081877F808378940E94860FF801AE
:1054C0001082F701808188608083CF70F801C083EB
:1054D000FF91EF91CF91BF91AF919F918F917F916C
:1054E0006F915F914F913F912F911F910F91FF907D
:1054F000EF900F900FBE0F901F901895AA1BBB1B2B
:1055000051E107C0AA1FBB1FA617B70710F0A61BC3
:10551000B70B881F991F5A95A9F780959095BC01E4
:10552000CD01089597FB072E16F4009406D077FD61
:1055300008D0E4DF07FC05D03EF4909581959F4F9D
:105540000895709561957F4F0895EE0FFF1F0590A8
:10555000F491E02D099469279627692778278727F2
:10556000782708952F923F924F925F926F927F9289
:105570008F929F92AF92BF92CF92DF92EF92FF9263
:105580000F931F93CF93DF93CDB7DEB7CA1BDB0B0F
:105590000FB6F894DEBF0FBECDBF09942A883988B4
:1055A00048885F846E847D848C849B84AA84B984BB
:1055B000C884DF80EE80FD800C811B81AA81B981C7
:1055C000CE0FD11D0FB6F894DEBF0FBECDBFED01DB
:1055D0000895FB01DC0102C005900D92415050403E
:1055E000D8F70895FB01DC0104C08D91019080196A
:1055F00021F441505040C8F7881B990B0895FB01D6
:10560000DC0102C001900D9241505040D8F708953E
:10561000DC0101C06D9341505040E0F70895F999C5
:10562000FECF92BD81BDF89A992780B50895A8E173
:10563000B0E042E050E02FC0DC01A40FB51F4150A4
:10564000504040F0CB01840F951F2E9105D0415062
:105650005040D8F70895262FF999FECF92BD81BD0D
:10566000F89A019700B4021639F01FBA20BD0FB6A0
:10567000F894FA9AF99A0FBE08950396272FECDF53
:10568000EADF252FE9DF242FE7CF0196272FE4DF7C
:10569000E2CFDC01CB01FC01F999FECF06C0F2BDDF
:1056A000E1BDF89A319600B40D9241505040B8F7E0
:1056B0000895F894FFCF560A5B0A5D0A620A720ADF
:1056C000720A720A720A720A720A720A720A640A08
:1056D000680A6B0A700A800A860A8A0A63108910AF
:1056E0008F1089108F10E11002118F1008121512FF
:1056F000F919FD19EF19F519011A051A091AF21A03
:10570000F21A601B601B041C211C101B101B261CA2
:10571000951CA61CA61C9A27B527BC27FA25FA2596
:10572000EE27FE271128522857287F289028A928DD
:10573000AC28E825EC251D26292634263F26E6251B
:10574000E625E625E62586274226452649267426AF
:08575000B026B326B526EA26B7
:1057580028081E0A8709F10C070D0C0D110DE80C1D
:10576800AF0001500114000001000101355BDCA20B
:10577800058C2C5C004422B684016201AC008A02CC
:10578800A302C30231333236F4F5F6F7C63435973F
:1057980066949091E200E900EA00B500B600B7000F
:1057A800CD008301CC008A019201940121022302D9
:1057B80024022502260227022A02B300B4006F0041
:1057C80070009F01CB019F02A002E200E900EA00FD
:1057D800B500B600B700CD008301CC008A01920164
:1057E80094012102230224022502260227022A020A
:1057F800B300B4006F0070009F01CB019F02A002AC
:00000001FF
